
 Start  Stop   Length Name               Class

 00000H 03272H 03273H _TEXT              CODE
 03273H 03317H 000A5H RACE_TEXT          CODE
 03318H 04926H 0160FH RACEMAIN_TEXT      CODE
 04927H 04C94H 0036EH ACTOR_TEXT         CODE
 04C95H 04E4CH 001B8H NEGO_TEXT          CODE
 04E50H 06ECFH 02080H NEGOFNT_TEXT       CODE
 06ED0H 06F51H 00082H GAMEUTIL_TEXT      CODE
 06F52H 070BBH 0016AH DISK_TEXT          CODE
 070BCH 071CAH 0010FH KEY_TEXT           CODE
 071CBH 077BDH 005F3H MCGA_TEXT          CODE
 077BEH 07844H 00087H ERROR_TEXT         CODE
 07845H 0827BH 00A37H FX4_TEXT           CODE
 08280H 08280H 00000H _FARDATA           FAR_DATA
 08280H 08280H 00000H _FARBSS            FAR_BSS
 08280H 08280H 00000H _OVERLAY_          OVRINFO
 08280H 08280H 00000H _1STUB_            STUBSEG
 08280H 0884BH 005CCH _DATA              DATA
 0884CH 0884DH 00002H _CVTSEG            DATA
 0884EH 08853H 00006H _SCNSEG            DATA
 08854H 08854H 00000H _CONST             CONST
 08854H 08865H 00012H _INIT_             INITDATA
 08866H 08866H 00000H _INITEND_          INITDATA
 08866H 08866H 00000H _EXIT_             EXITDATA
 08866H 08866H 00000H _EXITEND_          EXITDATA
 08866H 09869H 01004H _BSS               BSS
 0986AH 0986AH 00000H _BSSEND            BSSEND
 09870H 098EFH 00080H _STACK             STACK


Detailed map of segments

 0000:0000 0295 C=CODE   S=_TEXT          G=(none)  M=c0.ASM     ACBP=28
 0000:0295 002D C=CODE   S=_TEXT          G=(none)  M=ATEXIT     ACBP=28
 0000:02C2 0049 C=CODE   S=_TEXT          G=(none)  M=CLOCK      ACBP=28
 0000:030B 0000 C=CODE   S=_TEXT          G=(none)  M=CTYPE      ACBP=28
 0000:030B 003D C=CODE   S=_TEXT          G=(none)  M=DOSFATTR   ACBP=28
 0000:0348 0093 C=CODE   S=_TEXT          G=(none)  M=EXIT       ACBP=28
 0000:03DB 0000 C=CODE   S=_TEXT          G=(none)  M=FILES      ACBP=28
 0000:03DB 0000 C=CODE   S=_TEXT          G=(none)  M=FILES2     ACBP=28
 0000:03DB 0000 C=CODE   S=_TEXT          G=(none)  M=FMODE      ACBP=28
 0000:03DB 0026 C=CODE   S=_TEXT          G=(none)  M=GETDATE    ACBP=28
 0000:0401 0020 C=CODE   S=_TEXT          G=(none)  M=GETVECT    ACBP=28
 0000:0421 00AE C=CODE   S=_TEXT          G=(none)  M=H_LDIV     ACBP=28
 0000:04CF 0021 C=CODE   S=_TEXT          G=(none)  M=H_LLSH     ACBP=28
 0000:04F0 0088 C=CODE   S=_TEXT          G=(none)  M=H_PADA     ACBP=28
 0000:0578 0060 C=CODE   S=_TEXT          G=(none)  M=H_PADD     ACBP=28
 0000:05D8 004B C=CODE   S=_TEXT          G=(none)  M=IOERROR    ACBP=28
 0000:0623 0011 C=CODE   S=_TEXT          G=(none)  M=ISATTY     ACBP=28
 0000:0634 00A2 C=CODE   S=_TEXT          G=(none)  M=LONGTOA    ACBP=28
 0000:06D6 0029 C=CODE   S=_TEXT          G=(none)  M=LSEEK      ACBP=28
 0000:06FF 00B6 C=CODE   S=_TEXT          G=(none)  M=MKNAME     ACBP=28
 0000:07B5 0017 C=CODE   S=_TEXT          G=(none)  M=N_LXMUL    ACBP=28
 0000:07CC 0021 C=CODE   S=_TEXT          G=(none)  M=N_PCMP     ACBP=28
 0000:07ED 0037 C=CODE   S=_TEXT          G=(none)  M=RAND       ACBP=28
 0000:0824 002F C=CODE   S=_TEXT          G=(none)  M=READA      ACBP=28
 0000:0853 002A C=CODE   S=_TEXT          G=(none)  M=SETDATE    ACBP=28
 0000:087D 00BA C=CODE   S=_TEXT          G=(none)  M=SETUPIO    ACBP=28
 0000:0937 0098 C=CODE   S=_TEXT          G=(none)  M=STIME      ACBP=28
 0000:09CF 0000 C=CODE   S=_TEXT          G=(none)  M=STKLEN     ACBP=28
 0000:09CF 0018 C=CODE   S=_TEXT          G=(none)  M=UNLINK     ACBP=28
 0000:09E7 04DB C=CODE   S=_TEXT          G=(none)  M=VPRINTER   ACBP=28
 0000:0EC2 0034 C=CODE   S=_TEXT          G=(none)  M=_STPCPY    ACBP=28
 0000:0EF6 001F C=CODE   S=_TEXT          G=(none)  M=CVTFAK     ACBP=28
 0000:0F15 0432 C=CODE   S=_TEXT          G=(none)  M=FARHEAP    ACBP=28
 0000:1347 0140 C=CODE   S=_TEXT          G=(none)  M=FBRK       ACBP=28
 0000:1487 008E C=CODE   S=_TEXT          G=(none)  M=FCALLOC    ACBP=28
 0000:1515 0029 C=CODE   S=_TEXT          G=(none)  M=IOCTL      ACBP=28
 0000:153E 0012 C=CODE   S=_TEXT          G=(none)  M=KBHIT      ACBP=28
 0000:1550 0004 C=CODE   S=_TEXT          G=(none)  M=REALCVT    ACBP=28
 0000:1554 001C C=CODE   S=_TEXT          G=(none)  M=SETBLOCK   ACBP=28
 0000:1570 0058 C=CODE   S=_TEXT          G=(none)  M=SETENVP    ACBP=28
 0000:15C8 0086 C=CODE   S=_TEXT          G=(none)  M=ATOL       ACBP=28
 0000:164E 001D C=CODE   S=_TEXT          G=(none)  M=CHMODA     ACBP=28
 0000:166B 0028 C=CODE   S=_TEXT          G=(none)  M=CLOSE      ACBP=28
 0000:1693 001E C=CODE   S=_TEXT          G=(none)  M=CLOSEA     ACBP=28
 0000:16B1 007B C=CODE   S=_TEXT          G=(none)  M=CREATA     ACBP=28
 0000:172C 0077 C=CODE   S=_TEXT          G=(none)  M=EOF        ACBP=28
 0000:17A3 00B8 C=CODE   S=_TEXT          G=(none)  M=FCLOSE     ACBP=28
 0000:185B 00CD C=CODE   S=_TEXT          G=(none)  M=FFLUSH     ACBP=28
 0000:1928 0042 C=CODE   S=_TEXT          G=(none)  M=FLUSHALL   ACBP=28
 0000:196A 020C C=CODE   S=_TEXT          G=(none)  M=FOPEN      ACBP=28
 0000:1B76 0182 C=CODE   S=_TEXT          G=(none)  M=FREAD      ACBP=28
 0000:1CF8 01E2 C=CODE   S=_TEXT          G=(none)  M=FSEEK      ACBP=28
 0000:1EDA 01C8 C=CODE   S=_TEXT          G=(none)  M=GETC       ACBP=28
 0000:20A2 0070 C=CODE   S=_TEXT          G=(none)  M=GETENV     ACBP=28
 0000:2112 0024 C=CODE   S=_TEXT          G=(none)  M=MEMCPY     ACBP=28
 0000:2136 0043 C=CODE   S=_TEXT          G=(none)  M=MEMSET     ACBP=28
 0000:2179 019C C=CODE   S=_TEXT          G=(none)  M=OPEN       ACBP=28
 0000:2315 004F C=CODE   S=_TEXT          G=(none)  M=OPENA      ACBP=28
 0000:2364 001B C=CODE   S=_TEXT          G=(none)  M=PRINTF     ACBP=28
 0000:237F 03C8 C=CODE   S=_TEXT          G=(none)  M=PUTC       ACBP=28
 0000:2747 00D1 C=CODE   S=_TEXT          G=(none)  M=READ       ACBP=28
 0000:2818 0003 C=CODE   S=_TEXT          G=(none)  M=READU      ACBP=28
 0000:281B 011D C=CODE   S=_TEXT          G=(none)  M=SETVBUF    ACBP=28
 0000:2938 0083 C=CODE   S=_TEXT          G=(none)  M=SPRINTF    ACBP=28
 0000:29BB 003F C=CODE   S=_TEXT          G=(none)  M=STRCAT     ACBP=28
 0000:29FA 0029 C=CODE   S=_TEXT          G=(none)  M=STRCPY     ACBP=28
 0000:2A23 001F C=CODE   S=_TEXT          G=(none)  M=STRLEN     ACBP=28
 0000:2A42 0031 C=CODE   S=_TEXT          G=(none)  M=STRNCPY    ACBP=28
 0000:2A73 032E C=CODE   S=_TEXT          G=(none)  M=TIMECVT    ACBP=28
 0000:2DA1 02CD C=CODE   S=_TEXT          G=(none)  M=TZSET      ACBP=28
 0000:306E 0151 C=CODE   S=_TEXT          G=(none)  M=WRITE      ACBP=28
 0000:31BF 003C C=CODE   S=_TEXT          G=(none)  M=WRITEA     ACBP=28
 0000:31FB 0003 C=CODE   S=_TEXT          G=(none)  M=WRITEU     ACBP=28
 0000:31FE 003D C=CODE   S=_TEXT          G=(none)  M=XFCLOSE    ACBP=28
 0000:323B 0038 C=CODE   S=_TEXT          G=(none)  M=XFFLUSH    ACBP=28
 0327:0003 00A5 C=CODE   S=RACE_TEXT      G=(none)  M=RACE.C     ACBP=28
 0331:0008 160F C=CODE   S=RACEMAIN_TEXT  G=(none)  M=RACEMAIN.C ACBP=28
 0492:0007 036E C=CODE   S=ACTOR_TEXT     G=(none)  M=ACTOR.C    ACBP=28
 04C9:0005 01B8 C=CODE   S=NEGO_TEXT      G=(none)  M=NEGO.C     ACBP=28
 04E5:0000 2080 C=CODE   S=NEGOFNT_TEXT   G=(none)  M=::         ACBP=68
 06ED:0000 0082 C=CODE   S=GAMEUTIL_TEXT  G=(none)  M=GAMEUTIL   ACBP=28
 06F5:0002 016A C=CODE   S=DISK_TEXT      G=(none)  M=DISK       ACBP=28
 070B:000C 010F C=CODE   S=KEY_TEXT       G=(none)  M=KEY        ACBP=28
 071C:000B 05F3 C=CODE   S=MCGA_TEXT      G=(none)  M=MCGA       ACBP=28
 077B:000E 0087 C=CODE   S=ERROR_TEXT     G=(none)  M=ERROR      ACBP=28
 0784:0005 0A37 C=CODE   S=FX4_TEXT       G=(none)  M=FX4        ACBP=28
 0828:0000 0000 C=FAR_DATA S=_FARDATA       G=(none)  M=c0.ASM     ACBP=68
 0828:0000 0000 C=FAR_BSS S=_FARBSS        G=(none)  M=c0.ASM     ACBP=68
 0828:0000 0000 C=OVRINFO S=_OVERLAY_      G=(none)  M=c0.ASM     ACBP=68
 0828:0000 0000 C=STUBSEG S=_1STUB_        G=(none)  M=c0.ASM     ACBP=68
 0828:0000 0093 C=DATA   S=_DATA          G=DGROUP  M=c0.ASM     ACBP=68
 0828:0094 000A C=DATA   S=_DATA          G=DGROUP  M=RACE.C     ACBP=48
 0828:009E 0061 C=DATA   S=_DATA          G=DGROUP  M=RACEMAIN.C ACBP=48
 0828:0100 0035 C=DATA   S=_DATA          G=DGROUP  M=ACTOR.C    ACBP=48
 0828:0136 0001 C=DATA   S=_DATA          G=DGROUP  M=NEGO.C     ACBP=48
 0828:0138 0000 C=DATA   S=_DATA          G=DGROUP  M=GAMEUTIL   ACBP=48
 0828:0138 000A C=DATA   S=_DATA          G=DGROUP  M=DISK       ACBP=48
 0828:0142 0002 C=DATA   S=_DATA          G=DGROUP  M=KEY        ACBP=48
 0828:0144 0008 C=DATA   S=_DATA          G=DGROUP  M=MCGA       ACBP=48
 0828:014C 002B C=DATA   S=_DATA          G=DGROUP  M=ERROR      ACBP=48
 0828:0178 0031 C=DATA   S=_DATA          G=DGROUP  M=FX4        ACBP=48
 0828:01AA 0002 C=DATA   S=_DATA          G=DGROUP  M=ATEXIT     ACBP=48
 0828:01AC 0000 C=DATA   S=_DATA          G=DGROUP  M=CLOCK      ACBP=48
 0828:01AC 0101 C=DATA   S=_DATA          G=DGROUP  M=CTYPE      ACBP=48
 0828:02AE 0000 C=DATA   S=_DATA          G=DGROUP  M=DOSFATTR   ACBP=48
 0828:02AE 000C C=DATA   S=_DATA          G=DGROUP  M=EXIT       ACBP=48
 0828:02BA 0190 C=DATA   S=_DATA          G=DGROUP  M=FILES      ACBP=48
 0828:044A 002A C=DATA   S=_DATA          G=DGROUP  M=FILES2     ACBP=48
 0828:0474 0004 C=DATA   S=_DATA          G=DGROUP  M=FMODE      ACBP=48
 0828:0478 0000 C=DATA   S=_DATA          G=DGROUP  M=GETDATE    ACBP=48
 0828:0478 0000 C=DATA   S=_DATA          G=DGROUP  M=GETVECT    ACBP=48
 0828:0478 0000 C=DATA   S=_DATA          G=DGROUP  M=H_LDIV     ACBP=48
 0828:0478 0000 C=DATA   S=_DATA          G=DGROUP  M=H_LLSH     ACBP=48
 0828:0478 0000 C=DATA   S=_DATA          G=DGROUP  M=H_PADA     ACBP=48
 0828:0478 0000 C=DATA   S=_DATA          G=DGROUP  M=H_PADD     ACBP=48
 0828:0478 005B C=DATA   S=_DATA          G=DGROUP  M=IOERROR    ACBP=48
 0828:04D4 0000 C=DATA   S=_DATA          G=DGROUP  M=ISATTY     ACBP=48
 0828:04D4 0000 C=DATA   S=_DATA          G=DGROUP  M=LONGTOA    ACBP=48
 0828:04D4 0000 C=DATA   S=_DATA          G=DGROUP  M=LSEEK      ACBP=48
 0828:04D4 0009 C=DATA   S=_DATA          G=DGROUP  M=MKNAME     ACBP=48
 0828:04DE 0000 C=DATA   S=_DATA          G=DGROUP  M=N_LXMUL    ACBP=48
 0828:04DE 0000 C=DATA   S=_DATA          G=DGROUP  M=N_PCMP     ACBP=48
 0828:04DE 0004 C=DATA   S=_DATA          G=DGROUP  M=RAND       ACBP=48
 0828:04E2 0000 C=DATA   S=_DATA          G=DGROUP  M=READA      ACBP=48
 0828:04E2 0000 C=DATA   S=_DATA          G=DGROUP  M=SETDATE    ACBP=48
 0828:04E2 0000 C=DATA   S=_DATA          G=DGROUP  M=SETUPIO    ACBP=48
 0828:04E2 0000 C=DATA   S=_DATA          G=DGROUP  M=STIME      ACBP=48
 0828:04E2 0002 C=DATA   S=_DATA          G=DGROUP  M=STKLEN     ACBP=48
 0828:04E4 0000 C=DATA   S=_DATA          G=DGROUP  M=UNLINK     ACBP=48
 0828:04E4 0067 C=DATA   S=_DATA          G=DGROUP  M=VPRINTER   ACBP=48
 0828:054C 0000 C=DATA   S=_DATA          G=DGROUP  M=_STPCPY    ACBP=48
 0828:054C 0031 C=DATA   S=_DATA          G=DGROUP  M=CVTFAK     ACBP=48
 0828:057E 0000 C=DATA   S=_DATA          G=DGROUP  M=FARHEAP    ACBP=48
 0828:057E 0002 C=DATA   S=_DATA          G=DGROUP  M=FBRK       ACBP=48
 0828:0580 0000 C=DATA   S=_DATA          G=DGROUP  M=FCALLOC    ACBP=48
 0828:0580 0000 C=DATA   S=_DATA          G=DGROUP  M=IOCTL      ACBP=48
 0828:0580 0002 C=DATA   S=_DATA          G=DGROUP  M=KBHIT      ACBP=48
 0828:0582 0000 C=DATA   S=_DATA          G=DGROUP  M=REALCVT    ACBP=48
 0828:0582 0000 C=DATA   S=_DATA          G=DGROUP  M=SETBLOCK   ACBP=48
 0828:0582 0004 C=DATA   S=_DATA          G=DGROUP  M=SETENVP    ACBP=48
 0828:0586 0000 C=DATA   S=_DATA          G=DGROUP  M=ATOL       ACBP=48
 0828:0586 0000 C=DATA   S=_DATA          G=DGROUP  M=CHMODA     ACBP=48
 0828:0586 0000 C=DATA   S=_DATA          G=DGROUP  M=CLOSE      ACBP=48
 0828:0586 0000 C=DATA   S=_DATA          G=DGROUP  M=CLOSEA     ACBP=48
 0828:0586 0000 C=DATA   S=_DATA          G=DGROUP  M=CREATA     ACBP=48
 0828:0586 0000 C=DATA   S=_DATA          G=DGROUP  M=EOF        ACBP=48
 0828:0586 0000 C=DATA   S=_DATA          G=DGROUP  M=FCLOSE     ACBP=48
 0828:0586 0000 C=DATA   S=_DATA          G=DGROUP  M=FFLUSH     ACBP=48
 0828:0586 0000 C=DATA   S=_DATA          G=DGROUP  M=FLUSHALL   ACBP=48
 0828:0586 0000 C=DATA   S=_DATA          G=DGROUP  M=FOPEN      ACBP=48
 0828:0586 0000 C=DATA   S=_DATA          G=DGROUP  M=FREAD      ACBP=48
 0828:0586 0000 C=DATA   S=_DATA          G=DGROUP  M=FSEEK      ACBP=48
 0828:0586 0000 C=DATA   S=_DATA          G=DGROUP  M=GETC       ACBP=48
 0828:0586 0000 C=DATA   S=_DATA          G=DGROUP  M=GETENV     ACBP=48
 0828:0586 0000 C=DATA   S=_DATA          G=DGROUP  M=MEMCPY     ACBP=48
 0828:0586 0000 C=DATA   S=_DATA          G=DGROUP  M=MEMSET     ACBP=48
 0828:0586 0000 C=DATA   S=_DATA          G=DGROUP  M=OPEN       ACBP=48
 0828:0586 0000 C=DATA   S=_DATA          G=DGROUP  M=OPENA      ACBP=48
 0828:0586 0000 C=DATA   S=_DATA          G=DGROUP  M=PRINTF     ACBP=48
 0828:0586 0001 C=DATA   S=_DATA          G=DGROUP  M=PUTC       ACBP=48
 0828:0588 0000 C=DATA   S=_DATA          G=DGROUP  M=READ       ACBP=48
 0828:0588 0000 C=DATA   S=_DATA          G=DGROUP  M=READU      ACBP=48
 0828:0588 0004 C=DATA   S=_DATA          G=DGROUP  M=SETVBUF    ACBP=48
 0828:058C 0000 C=DATA   S=_DATA          G=DGROUP  M=SPRINTF    ACBP=48
 0828:058C 0000 C=DATA   S=_DATA          G=DGROUP  M=STRCAT     ACBP=48
 0828:058C 0000 C=DATA   S=_DATA          G=DGROUP  M=STRCPY     ACBP=48
 0828:058C 0000 C=DATA   S=_DATA          G=DGROUP  M=STRLEN     ACBP=48
 0828:058C 0000 C=DATA   S=_DATA          G=DGROUP  M=STRNCPY    ACBP=48
 0828:058C 000C C=DATA   S=_DATA          G=DGROUP  M=TIMECVT    ACBP=48
 0828:0598 0033 C=DATA   S=_DATA          G=DGROUP  M=TZSET      ACBP=48
 0828:05CC 0000 C=DATA   S=_DATA          G=DGROUP  M=WRITE      ACBP=48
 0828:05CC 0000 C=DATA   S=_DATA          G=DGROUP  M=WRITEA     ACBP=48
 0828:05CC 0000 C=DATA   S=_DATA          G=DGROUP  M=WRITEU     ACBP=48
 0828:05CC 0000 C=DATA   S=_DATA          G=DGROUP  M=XFCLOSE    ACBP=48
 0828:05CC 0000 C=DATA   S=_DATA          G=DGROUP  M=XFFLUSH    ACBP=48
 0828:05CC 0000 C=DATA   S=_CVTSEG        G=DGROUP  M=c0.ASM     ACBP=48
 0828:05CC 0002 C=DATA   S=_CVTSEG        G=DGROUP  M=CVTFAK     ACBP=48
 0828:05CE 0000 C=DATA   S=_CVTSEG        G=DGROUP  M=REALCVT    ACBP=48
 0828:05CE 0000 C=DATA   S=_SCNSEG        G=DGROUP  M=c0.ASM     ACBP=48
 0828:05CE 0006 C=DATA   S=_SCNSEG        G=DGROUP  M=CVTFAK     ACBP=48
 0828:05D4 0000 C=CONST  S=_CONST         G=DGROUP  M=c0.ASM     ACBP=48
 0828:05D4 0000 C=INITDATA S=_INIT_         G=DGROUP  M=c0.ASM     ACBP=48
 0828:05D4 0006 C=INITDATA S=_INIT_         G=DGROUP  M=SETUPIO    ACBP=48
 0828:05DA 0006 C=INITDATA S=_INIT_         G=DGROUP  M=SETENVP    ACBP=48
 0828:05E0 0006 C=INITDATA S=_INIT_         G=DGROUP  M=TZSET      ACBP=48
 0828:05E6 0000 C=INITDATA S=_INITEND_      G=DGROUP  M=c0.ASM     ACBP=28
 0828:05E6 0000 C=EXITDATA S=_EXIT_         G=DGROUP  M=c0.ASM     ACBP=48
 0828:05E6 0000 C=EXITDATA S=_EXITEND_      G=DGROUP  M=c0.ASM     ACBP=28
 0828:05E6 0000 C=BSS    S=_BSS           G=DGROUP  M=c0.ASM     ACBP=48
 0828:05E6 0300 C=BSS    S=_BSS           G=DGROUP  M=RACE.C     ACBP=48
 0828:08E6 032C C=BSS    S=_BSS           G=DGROUP  M=RACEMAIN.C ACBP=48
 0828:0C12 00CC C=BSS    S=_BSS           G=DGROUP  M=ACTOR.C    ACBP=48
 0828:0CDE 0000 C=BSS    S=_BSS           G=DGROUP  M=NEGO.C     ACBP=48
 0828:0CDE 0000 C=BSS    S=_BSS           G=DGROUP  M=GAMEUTIL   ACBP=48
 0828:0CDE 0000 C=BSS    S=_BSS           G=DGROUP  M=DISK       ACBP=48
 0828:0CDE 0104 C=BSS    S=_BSS           G=DGROUP  M=KEY        ACBP=48
 0828:0DE2 007C C=BSS    S=_BSS           G=DGROUP  M=MCGA       ACBP=48
 0828:0E5E 0004 C=BSS    S=_BSS           G=DGROUP  M=ERROR      ACBP=48
 0828:0E62 06EB C=BSS    S=_BSS           G=DGROUP  M=FX4        ACBP=48
 0828:154E 0080 C=BSS    S=_BSS           G=DGROUP  M=ATEXIT     ACBP=48
 0828:15CE 0001 C=BSS    S=_BSS           G=DGROUP  M=CLOCK      ACBP=48
 0828:15D0 0000 C=BSS    S=_BSS           G=DGROUP  M=DOSFATTR   ACBP=48
 0828:15D0 0000 C=BSS    S=_BSS           G=DGROUP  M=GETVECT    ACBP=48
 0828:15D0 0000 C=BSS    S=_BSS           G=DGROUP  M=IOERROR    ACBP=48
 0828:15D0 0000 C=BSS    S=_BSS           G=DGROUP  M=ISATTY     ACBP=48
 0828:15D0 0000 C=BSS    S=_BSS           G=DGROUP  M=LONGTOA    ACBP=48
 0828:15D0 0000 C=BSS    S=_BSS           G=DGROUP  M=LSEEK      ACBP=48
 0828:15D0 000D C=BSS    S=_BSS           G=DGROUP  M=MKNAME     ACBP=48
 0828:15DE 0000 C=BSS    S=_BSS           G=DGROUP  M=READA      ACBP=48
 0828:15DE 0000 C=BSS    S=_BSS           G=DGROUP  M=SETDATE    ACBP=48
 0828:15DE 0000 C=BSS    S=_BSS           G=DGROUP  M=SETUPIO    ACBP=48
 0828:15DE 0000 C=BSS    S=_BSS           G=DGROUP  M=UNLINK     ACBP=48
 0828:15DE 0000 C=BSS    S=_BSS           G=DGROUP  M=VPRINTER   ACBP=48
 0828:15DE 0000 C=BSS    S=_BSS           G=DGROUP  M=FCALLOC    ACBP=48
 0828:15DE 0000 C=BSS    S=_BSS           G=DGROUP  M=IOCTL      ACBP=48
 0828:15DE 0000 C=BSS    S=_BSS           G=DGROUP  M=KBHIT      ACBP=48
 0828:15DE 0000 C=BSS    S=_BSS           G=DGROUP  M=SETBLOCK   ACBP=48
 0828:15DE 0000 C=BSS    S=_BSS           G=DGROUP  M=ATOL       ACBP=48
 0828:15DE 0000 C=BSS    S=_BSS           G=DGROUP  M=CHMODA     ACBP=48
 0828:15DE 0000 C=BSS    S=_BSS           G=DGROUP  M=CLOSEA     ACBP=48
 0828:15DE 0000 C=BSS    S=_BSS           G=DGROUP  M=CREATA     ACBP=48
 0828:15DE 0000 C=BSS    S=_BSS           G=DGROUP  M=EOF        ACBP=48
 0828:15DE 0000 C=BSS    S=_BSS           G=DGROUP  M=FREAD      ACBP=48
 0828:15DE 0001 C=BSS    S=_BSS           G=DGROUP  M=GETC       ACBP=48
 0828:15E0 0000 C=BSS    S=_BSS           G=DGROUP  M=GETENV     ACBP=48
 0828:15E0 0000 C=BSS    S=_BSS           G=DGROUP  M=MEMCPY     ACBP=48
 0828:15E0 0000 C=BSS    S=_BSS           G=DGROUP  M=MEMSET     ACBP=48
 0828:15E0 0000 C=BSS    S=_BSS           G=DGROUP  M=OPEN       ACBP=48
 0828:15E0 0000 C=BSS    S=_BSS           G=DGROUP  M=OPENA      ACBP=48
 0828:15E0 0001 C=BSS    S=_BSS           G=DGROUP  M=PUTC       ACBP=48
 0828:15E2 0000 C=BSS    S=_BSS           G=DGROUP  M=READ       ACBP=48
 0828:15E2 0000 C=BSS    S=_BSS           G=DGROUP  M=STRCAT     ACBP=48
 0828:15E2 0000 C=BSS    S=_BSS           G=DGROUP  M=STRCPY     ACBP=48
 0828:15E2 0000 C=BSS    S=_BSS           G=DGROUP  M=STRLEN     ACBP=48
 0828:15E2 0000 C=BSS    S=_BSS           G=DGROUP  M=STRNCPY    ACBP=48
 0828:15E2 0008 C=BSS    S=_BSS           G=DGROUP  M=TZSET      ACBP=48
 0828:15EA 0000 C=BSS    S=_BSS           G=DGROUP  M=WRITEA     ACBP=48
 0828:15EA 0000 C=BSSEND S=_BSSEND        G=DGROUP  M=c0.ASM     ACBP=28
 0987:0000 0080 C=STACK  S=_STACK         G=(none)  M=c0.ASM     ACBP=74

  Address         Publics by Name

 0828:0000 idle  DATASEG@
 0000:0291 idle  DGROUP@
 0000:0424 idle  F_LDIV@
 0000:0433 idle  F_LMOD@
 0000:042B idle  F_LUDIV@
 0000:043B idle  F_LUMOD@
 0000:04D2 idle  F_LXLSH@
 0000:04F3 idle  F_PADA@
 0000:057B idle  F_PADD@
 0000:0537 idle  F_PSBA@
 0000:05AA idle  F_PSUB@
 0000:0424 idle  LDIV@
 0000:0433 idle  LMOD@
 0000:042B idle  LUDIV@
 0000:043B idle  LUMOD@
 0000:04D2 idle  LXLSH@
 0000:0421       N_LDIV@
 0000:0430       N_LMOD@
 0000:0428 idle  N_LUDIV@
 0000:0438 idle  N_LUMOD@
 0000:04CF       N_LXLSH@
 0000:07B5       N_LXMUL@
 0000:04F0       N_PADA@
 0000:0578       N_PADD@
 0000:07CC       N_PCMP@
 0000:0534 idle  N_PSBA@
 0000:05A7 idle  N_PSUB@
 0000:04F3 idle  PADA@
 0000:057B idle  PADD@
 0000:0537 idle  PSBA@
 0000:05AA idle  PSUB@
 0000:027A       _abort
 06ED:0000       _AllocMemory
 0000:0295 idle  _atexit
 0000:163D idle  _atoi
 0000:15C8       _atol
 071C:03CB idle  _CellophaneBox
 0828:0F66       _cellophaneFlag
 0828:0F62       _cellophanePalette
 0784:0708 idle  _CFX4Put_Sprite0
 0784:0960 idle  _CFX4Put_Sprite0S
 0784:0651 idle  _CFX4Put_Sprite1
 0784:0891 idle  _CFX4Put_Sprite1S
 0784:0005 idle  _ChangeCellophane
 0331:158A       _chickRace
 070B:00FB       _ClearKBD
 071C:05EB idle  _ClearPage
 0828:017C idle  _Clip_EX
 0828:017E idle  _Clip_EY
 0828:0178 idle  _Clip_SX
 0828:017A idle  _Clip_SY
 0000:02C2       _clock
 0000:166B       _close
 06F5:014D idle  _CloseDisk
 0331:0CED idle  _congrRace
 071C:05BD       _CopyPage
 071C:05D5 idle  _CopyScreen
 0000:1711       _creatnew
 0000:16F6 idle  _creattemp
 0828:05BE       _daylight
 070B:0048       _DeinitKBD
 0828:0E5E idle  _Deinit_system
 0492:0058       _delActor
 0828:0E4E       _displayP
 0000:2A73       _dostounix
 0492:00C2       _endFrameActor
 0828:0582       _environ
 0000:172C       _eof
 0828:007F       _errno
 077B:0028       _Errorexit
 077B:0051       _Errorexitf
 0000:03A0       _exit
 071C:01B4 idle  _FadeIn
 071C:02BF idle  _FadeOut
 0000:1487       _farcalloc
 0000:1055       _farfree
 0000:1169       _farmalloc
 0000:12CD idle  _farrealloc
 0000:17A3       _fclose
 0000:185B       _fflush
 0000:1FA8       _fgetc
 0000:2096 idle  _fgetchar
 071C:049E idle  _fillbox13
 0000:1928       _flushall
 0000:1B41       _fopen
 0000:239B idle  _fputc
 0000:2530 idle  _fputchar
 0000:1C6A       _fread
 0000:1055       _free
 0784:0233       _Free_FX4
 0000:1D7A       _fseek
 0000:1DFA idle  _ftell
 0784:0607 idle  _FX4Put_Sprite0
 0784:082B idle  _FX4Put_Sprite0S
 0784:05C5 idle  _FX4Put_Sprite1
 0784:07CC idle  _FX4Put_Sprite1S
 0492:0111       _getCutActor
 0000:03DB       _getdate
 0492:012E       _getDirActor
 0000:20A2       _getenv
 0492:00DC idle  _getMoveXActor
 0492:00F6 idle  _getMoveYActor
 0000:03EE       _gettime
 0000:0401       _getvect
 0784:00A2       _InitCellophaneColor
 0331:14B1 idle  _initChick
 04C9:0005 idle  _InitializeNego
 077B:000E       _Initialize_Error
 071C:04DF       _Initialize_Mcga
 070B:000C       _InitKBD
 071C:0409 idle  _InitPaletteScroll
 0492:01E4       _initPattern
 0327:0051 idle  _initRace
 071C:04D5       _Init_mode
 0000:1515       _ioctl
 0000:0623       _isatty
 0828:0F67 idle  _ITEM4
 0000:153E       _kbhit
 070B:00D6 idle  _Keyboardwait
 0828:0142 idle  _KeyIntFlag
 070B:0071 idle  _keyStatusCheck
 0327:0003 idle  _loadPalette
 0784:00E2       _Load_FX4
 0000:06D6       _lseek
 06F5:011D idle  _LseekDisk
 0327:007D       _main
 0000:115F       _malloc
 0000:2112       _memcpy
 0000:215A       _memset
 071C:0570 idle  _Mode320x200
 071C:0549 idle  _ModeX
 04E5:0000       _negodat
 04C9:017E idle  _negoprintf
 0492:0007       _newActor
 0492:0198       _nextFrameActor
 0828:0CDE idle  _oldKBD
 0000:21A6       _open
 06F5:0002       _OpenforLoad
 06F5:0039 idle  _OpenforSave
 071C:0467 idle  _PaletteScroll
 0828:0DE2 idle  _palscrbuf
 0828:0E42 idle  _palscrEB
 0828:0E44 idle  _palscrSB
 0828:0E46 idle  _palscrSC
 0000:2364       _printf
 0492:014B       _processActor
 0828:0E4A       _processP
 0492:01BA       _putActor
 071C:000B       _PutHMGImage13C
 0784:0295       _Put_FX4
 0331:1568 idle  _quitChick
 0492:0322       _quitPattern
 0327:006D idle  _quitRace
 0000:07FE       _rand
 0000:2818       _read
 06F5:0082 idle  _ReadDisk
 071C:00F8 idle  _Readpalette
 0331:0C78 idle  _readyRace
 0000:12C6 idle  _realloc
 0331:0D8B idle  _runRace
 0492:0069       _setActionActor
 0000:1554       _setblock
 0784:001A idle  _SetCellophaneColor
 0000:0853       _setdate
 0000:2136       _setmem
 04C9:0173       _setNegoBack
 071C:058C       _SetPage
 071C:014E       _Setpalette
 071C:0194 idle  _Setpalettenosnow
 071C:0133 idle  _Setsinglecolor
 0000:0868       _settime
 0000:281B       _setvbuf
 0000:0410       _setvect
 0000:2978 idle  _sprintf
 0000:07ED       _srand
 0000:0937 idle  _stime
 0000:29BB       _strcat
 0000:29FA       _strcpy
 0000:2A23       _strlen
 0000:2A42       _strncpy
 0000:0977       _time
 0828:05BA       _timezone
 0828:0E62 idle  _totalCellophaneColor
 0828:05B2 idle  _tzname
 0000:2DA1       _tzset
 0000:2B9D       _unixtodos
 0000:09CF       _unlink
 0000:299A       _vsprintf
 06ED:004C idle  _WaitTime
 0000:31FB       _write
 06F5:00A8 idle  _WriteDisk
 06F5:00CE idle  _WriteDiskF
 0828:0E52       __activepage
 0000:1000 idle  __AHINCR
 0000:000C idle  __AHSHIFT
 0828:01AA       __atexitcnt
 0828:154E       __atexittbl
 0828:0E48       __backgroundcolor
 0000:13BD       __brk
 0828:008B       __brklvl
 0828:006B idle  __C0argc
 0828:006D idle  __C0argv
 0828:0071       __C0environ
 0828:0581 idle  __cChar
 0000:03C1 idle  __cexit
 0828:0580 idle  __cFlag
 0000:016A       __checknull
 0000:164E       __chmod
 0000:0157       __cleanup
 0000:1693       __close
 0000:16DE       __creat
 0828:01AC       __ctype
 0000:0000  Abs  __cvtfak
 0000:03CF idle  __c_exit
 0828:0478       __doserrno
 0000:0611       __DOSERROR
 0828:047A idle  __dosErrorToSV
 0000:030B       __dos_getfileattr
 0000:032B idle  __dos_setfileattr
 0828:0075       __envLng
 0828:0077       __envseg
 0828:0079       __envSize
 0000:03AF       __exit
 0828:02AE       __exitbuf
 0828:02B2       __exitfopen
 0828:02B6 idle  __exitopen
 0000:1F90       __fgetc
 0828:0474       __fmode
 0828:0E49       __foregroundcolor
 0000:237F idle  __fputc
 0000:2544       __FPUTN
 0000:1AF7 idle  __GETFP
 0828:0087       __heapbase
 0828:008F       __heaptop
 0828:005B idle  __Int0Vector
 0828:005F idle  __Int4Vector
 0828:0063 idle  __Int5Vector
 0828:0067 idle  __Int6Vector
 0000:05D8       __IOERROR
 0000:2F8F       __ISDST
 0828:0143 idle  __KBHIT
 0828:0CE2       __KE
 0828:0D62       __KS
 0000:0634       __LONGTOA
 0331:0B87 idle  __loverChick
 0828:00A0 idle  __luckyTable
 0828:0146 idle  __mcgabottom
 0828:0148 idle  __mcgaleft
 0828:0E56 idle  __mcgapage
 0828:014A idle  __mcgaright
 0828:0144 idle  __mcgatop
 0000:06FF       __MKNAME
 0000:0293 idle  __MMODEL
 0828:0598 idle  __monthDay
 04C9:00A6 idle  __negoPutch
 04C9:0006 idle  __negoPutImage
 04C9:004D idle  __negoPutImageT
 04C9:00CD idle  __negoPuts
 0000:1FA5 idle  __Nfgetc
 0828:044A       __nfile
 0828:0476       __notUmask
 0000:2315       __open
 0828:044C       __openfd
 0000:1A26 idle  __OPENFP
 0828:007D idle  __osmajor
 0828:007E idle  __osminor
 0828:007D idle  __osversion
 0828:0E47 idle  __paletteDegree
 0331:0B2B idle  __processCongrChick
 0331:0AB8 idle  __processReadyChick
 0828:007B       __psp
 0331:09AA idle  __putHeartChick
 0000:0824       __read
 0000:1550       __REALCVT
 0828:05CC       __RealCvtVector
 0331:04C0 idle  __removeLooker
 0000:01C0       __restorezero
 0000:13FC       __sbrk
 0828:05CE idle  __ScanTodVector
 0331:082A idle  __selectActionChick
 0331:06B3 idle  __setBadChick
 0000:0000 idle  __setenvp__
 0331:065D idle  __setGoodChick
 0331:079F idle  __setNormalChick
 0000:087D       __setupio
 0828:0081       __StartTime
 0828:04E2       __stklen
 0000:0EC2       __stpcpy
 0828:02BA       __streams
 0000:016B       __terminate
 0000:075C idle  __TMPNAM
 0000:06B6       __UTOA
 0828:007D idle  __version
 0000:09FF       __VPRINTER
 0000:31BF       __write
 0000:31FE       __xfclose
 0000:323B       __xfflush
 0828:0085 idle  ___brklvl
 0000:0F15 idle  ___first
 0000:0F17 idle  ___last
 0000:2747       ___read
 0000:0F19 idle  ___rover
 0000:306E       ___write

  Address         Publics by Value

 0000:0000  Abs  __cvtfak
 0000:0000 idle  __setenvp__
 0000:000C idle  __AHSHIFT
 0000:0157       __cleanup
 0000:016A       __checknull
 0000:016B       __terminate
 0000:01C0       __restorezero
 0000:027A       _abort
 0000:0291 idle  DGROUP@
 0000:0293 idle  __MMODEL
 0000:0295 idle  _atexit
 0000:02C2       _clock
 0000:030B       __dos_getfileattr
 0000:032B idle  __dos_setfileattr
 0000:03A0       _exit
 0000:03AF       __exit
 0000:03C1 idle  __cexit
 0000:03CF idle  __c_exit
 0000:03DB       _getdate
 0000:03EE       _gettime
 0000:0401       _getvect
 0000:0410       _setvect
 0000:0421       N_LDIV@
 0000:0424 idle  F_LDIV@
 0000:0424 idle  LDIV@
 0000:0428 idle  N_LUDIV@
 0000:042B idle  F_LUDIV@
 0000:042B idle  LUDIV@
 0000:0430       N_LMOD@
 0000:0433 idle  F_LMOD@
 0000:0433 idle  LMOD@
 0000:0438 idle  N_LUMOD@
 0000:043B idle  LUMOD@
 0000:043B idle  F_LUMOD@
 0000:04CF       N_LXLSH@
 0000:04D2 idle  LXLSH@
 0000:04D2 idle  F_LXLSH@
 0000:04F0       N_PADA@
 0000:04F3 idle  F_PADA@
 0000:04F3 idle  PADA@
 0000:0534 idle  N_PSBA@
 0000:0537 idle  PSBA@
 0000:0537 idle  F_PSBA@
 0000:0578       N_PADD@
 0000:057B idle  F_PADD@
 0000:057B idle  PADD@
 0000:05A7 idle  N_PSUB@
 0000:05AA idle  F_PSUB@
 0000:05AA idle  PSUB@
 0000:05D8       __IOERROR
 0000:0611       __DOSERROR
 0000:0623       _isatty
 0000:0634       __LONGTOA
 0000:06B6       __UTOA
 0000:06D6       _lseek
 0000:06FF       __MKNAME
 0000:075C idle  __TMPNAM
 0000:07B5       N_LXMUL@
 0000:07CC       N_PCMP@
 0000:07ED       _srand
 0000:07FE       _rand
 0000:0824       __read
 0000:0853       _setdate
 0000:0868       _settime
 0000:087D       __setupio
 0000:0937 idle  _stime
 0000:0977       _time
 0000:09CF       _unlink
 0000:09FF       __VPRINTER
 0000:0EC2       __stpcpy
 0000:0F15 idle  ___first
 0000:0F17 idle  ___last
 0000:0F19 idle  ___rover
 0000:1000 idle  __AHINCR
 0000:1055       _farfree
 0000:1055       _free
 0000:115F       _malloc
 0000:1169       _farmalloc
 0000:12C6 idle  _realloc
 0000:12CD idle  _farrealloc
 0000:13BD       __brk
 0000:13FC       __sbrk
 0000:1487       _farcalloc
 0000:1515       _ioctl
 0000:153E       _kbhit
 0000:1550       __REALCVT
 0000:1554       _setblock
 0000:15C8       _atol
 0000:163D idle  _atoi
 0000:164E       __chmod
 0000:166B       _close
 0000:1693       __close
 0000:16DE       __creat
 0000:16F6 idle  _creattemp
 0000:1711       _creatnew
 0000:172C       _eof
 0000:17A3       _fclose
 0000:185B       _fflush
 0000:1928       _flushall
 0000:1A26 idle  __OPENFP
 0000:1AF7 idle  __GETFP
 0000:1B41       _fopen
 0000:1C6A       _fread
 0000:1D7A       _fseek
 0000:1DFA idle  _ftell
 0000:1F90       __fgetc
 0000:1FA5 idle  __Nfgetc
 0000:1FA8       _fgetc
 0000:2096 idle  _fgetchar
 0000:20A2       _getenv
 0000:2112       _memcpy
 0000:2136       _setmem
 0000:215A       _memset
 0000:21A6       _open
 0000:2315       __open
 0000:2364       _printf
 0000:237F idle  __fputc
 0000:239B idle  _fputc
 0000:2530 idle  _fputchar
 0000:2544       __FPUTN
 0000:2747       ___read
 0000:2818       _read
 0000:281B       _setvbuf
 0000:2978 idle  _sprintf
 0000:299A       _vsprintf
 0000:29BB       _strcat
 0000:29FA       _strcpy
 0000:2A23       _strlen
 0000:2A42       _strncpy
 0000:2A73       _dostounix
 0000:2B9D       _unixtodos
 0000:2DA1       _tzset
 0000:2F8F       __ISDST
 0000:306E       ___write
 0000:31BF       __write
 0000:31FB       _write
 0000:31FE       __xfclose
 0000:323B       __xfflush
 0327:0003 idle  _loadPalette
 0327:0051 idle  _initRace
 0327:006D idle  _quitRace
 0327:007D       _main
 0331:04C0 idle  __removeLooker
 0331:065D idle  __setGoodChick
 0331:06B3 idle  __setBadChick
 0331:079F idle  __setNormalChick
 0331:082A idle  __selectActionChick
 0331:09AA idle  __putHeartChick
 0331:0AB8 idle  __processReadyChick
 0331:0B2B idle  __processCongrChick
 0331:0B87 idle  __loverChick
 0331:0C78 idle  _readyRace
 0331:0CED idle  _congrRace
 0331:0D8B idle  _runRace
 0331:14B1 idle  _initChick
 0331:1568 idle  _quitChick
 0331:158A       _chickRace
 0492:0007       _newActor
 0492:0058       _delActor
 0492:0069       _setActionActor
 0492:00C2       _endFrameActor
 0492:00DC idle  _getMoveXActor
 0492:00F6 idle  _getMoveYActor
 0492:0111       _getCutActor
 0492:012E       _getDirActor
 0492:014B       _processActor
 0492:0198       _nextFrameActor
 0492:01BA       _putActor
 0492:01E4       _initPattern
 0492:0322       _quitPattern
 04C9:0005 idle  _InitializeNego
 04C9:0006 idle  __negoPutImage
 04C9:004D idle  __negoPutImageT
 04C9:00A6 idle  __negoPutch
 04C9:00CD idle  __negoPuts
 04C9:0173       _setNegoBack
 04C9:017E idle  _negoprintf
 04E5:0000       _negodat
 06ED:0000       _AllocMemory
 06ED:004C idle  _WaitTime
 06F5:0002       _OpenforLoad
 06F5:0039 idle  _OpenforSave
 06F5:0082 idle  _ReadDisk
 06F5:00A8 idle  _WriteDisk
 06F5:00CE idle  _WriteDiskF
 06F5:011D idle  _LseekDisk
 06F5:014D idle  _CloseDisk
 070B:000C       _InitKBD
 070B:0048       _DeinitKBD
 070B:0071 idle  _keyStatusCheck
 070B:00D6 idle  _Keyboardwait
 070B:00FB       _ClearKBD
 071C:000B       _PutHMGImage13C
 071C:00F8 idle  _Readpalette
 071C:0133 idle  _Setsinglecolor
 071C:014E       _Setpalette
 071C:0194 idle  _Setpalettenosnow
 071C:01B4 idle  _FadeIn
 071C:02BF idle  _FadeOut
 071C:03CB idle  _CellophaneBox
 071C:0409 idle  _InitPaletteScroll
 071C:0467 idle  _PaletteScroll
 071C:049E idle  _fillbox13
 071C:04D5       _Init_mode
 071C:04DF       _Initialize_Mcga
 071C:0549 idle  _ModeX
 071C:0570 idle  _Mode320x200
 071C:058C       _SetPage
 071C:05BD       _CopyPage
 071C:05D5 idle  _CopyScreen
 071C:05EB idle  _ClearPage
 077B:000E       _Initialize_Error
 077B:0028       _Errorexit
 077B:0051       _Errorexitf
 0784:0005 idle  _ChangeCellophane
 0784:001A idle  _SetCellophaneColor
 0784:00A2       _InitCellophaneColor
 0784:00E2       _Load_FX4
 0784:0233       _Free_FX4
 0784:0295       _Put_FX4
 0784:05C5 idle  _FX4Put_Sprite1
 0784:0607 idle  _FX4Put_Sprite0
 0784:0651 idle  _CFX4Put_Sprite1
 0784:0708 idle  _CFX4Put_Sprite0
 0784:07CC idle  _FX4Put_Sprite1S
 0784:082B idle  _FX4Put_Sprite0S
 0784:0891 idle  _CFX4Put_Sprite1S
 0784:0960 idle  _CFX4Put_Sprite0S
 0828:0000 idle  DATASEG@
 0828:005B idle  __Int0Vector
 0828:005F idle  __Int4Vector
 0828:0063 idle  __Int5Vector
 0828:0067 idle  __Int6Vector
 0828:006B idle  __C0argc
 0828:006D idle  __C0argv
 0828:0071       __C0environ
 0828:0075       __envLng
 0828:0077       __envseg
 0828:0079       __envSize
 0828:007B       __psp
 0828:007D idle  __osversion
 0828:007D idle  __osmajor
 0828:007D idle  __version
 0828:007E idle  __osminor
 0828:007F       _errno
 0828:0081       __StartTime
 0828:0085 idle  ___brklvl
 0828:0087       __heapbase
 0828:008B       __brklvl
 0828:008F       __heaptop
 0828:00A0 idle  __luckyTable
 0828:0142 idle  _KeyIntFlag
 0828:0143 idle  __KBHIT
 0828:0144 idle  __mcgatop
 0828:0146 idle  __mcgabottom
 0828:0148 idle  __mcgaleft
 0828:014A idle  __mcgaright
 0828:0178 idle  _Clip_SX
 0828:017A idle  _Clip_SY
 0828:017C idle  _Clip_EX
 0828:017E idle  _Clip_EY
 0828:01AA       __atexitcnt
 0828:01AC       __ctype
 0828:02AE       __exitbuf
 0828:02B2       __exitfopen
 0828:02B6 idle  __exitopen
 0828:02BA       __streams
 0828:044A       __nfile
 0828:044C       __openfd
 0828:0474       __fmode
 0828:0476       __notUmask
 0828:0478       __doserrno
 0828:047A idle  __dosErrorToSV
 0828:04E2       __stklen
 0828:0580 idle  __cFlag
 0828:0581 idle  __cChar
 0828:0582       _environ
 0828:0598 idle  __monthDay
 0828:05B2 idle  _tzname
 0828:05BA       _timezone
 0828:05BE       _daylight
 0828:05CC       __RealCvtVector
 0828:05CE idle  __ScanTodVector
 0828:0CDE idle  _oldKBD
 0828:0CE2       __KE
 0828:0D62       __KS
 0828:0DE2 idle  _palscrbuf
 0828:0E42 idle  _palscrEB
 0828:0E44 idle  _palscrSB
 0828:0E46 idle  _palscrSC
 0828:0E47 idle  __paletteDegree
 0828:0E48       __backgroundcolor
 0828:0E49       __foregroundcolor
 0828:0E4A       _processP
 0828:0E4E       _displayP
 0828:0E52       __activepage
 0828:0E56 idle  __mcgapage
 0828:0E5E idle  _Deinit_system
 0828:0E62 idle  _totalCellophaneColor
 0828:0F62       _cellophanePalette
 0828:0F66       _cellophaneFlag
 0828:0F67 idle  _ITEM4
 0828:154E       __atexittbl

Program entry point at 0000:0000

